:020000020000FC
:10000000FFC0E8C1E8C1E8C1E8C1E8C139C21EC209
:100010001EC21EC21AC2E6C116C216C2E0C1E0C1AB
:10002000E0C12FC216C226C226C22CC228C226C2D6
:040030002AC22AC2F4
:10020000F89400E810E000936100109361000EE1A3
:1002100005B901E204B904E408B90FEB07B900E03D
:100220000BB90EEF0AB9B1E0A0E0D5E0C0E000E004
:100230000D93BD17E9F7AC17D9F714E00FEF1EBF08
:100240000DBF00E005BF03E00CBB00E105BB01E210
:1002500004BD02E005BD00E006BD00E007BD00E012
:1002600008BD00E003BD00E0009380000DE00093B6
:10027000810000E00093820010E000E01093850010
:10028000009384001CE10DE1109389000093880025
:1002900010E000E010938B0000938A0010E000E073
:1002A000109387000093860000E107BB01E20093F2
:1002B000B00002E00093B10000E00093B20000E063
:1002C0000093B30000E00093B40000E00093B60098
:1002D00007E200937C0007EE00937A0000E00093B1
:1002E0007B0000E000937E0000E80093300000E017
:1002F00000937F0010E003E01093C5000093C4005A
:1003000000E20093C00008ED0093C10006E00093F6
:10031000C20000E000937B0000E000936900A89514
:1003200008E10093600009E20093600000E00093A0
:10033000640000E00DBB00E00093680000E0009363
:100340006B0000E000936C0000E000936D0000E0A3
:1003500000936E0002E000936F0000E000937000D5
:1003600090E003E0002EB1E0A0E27894A89590FF21
:1003700030C09E7F00912101063411F45C9A04C0C4
:10038000023411F45C9800C02091220110912301E5
:10039000009124017AD00093B40000912501063425
:1003A00011F45E9A04C0023411F45E9800C02091EA
:1003B0002601109127010091280167D008BD009106
:1003C0002A01013311F4409A04C0003311F440981B
:1003D00000C0CCCF189518951895189518951895B4
:1003E00018951895FFB60F931F932F9310E01C9B41
:1003F00011601B9B1260103011F42DE40CC0113001
:1004000011F420E608C0123011F427E704C01330BD
:1004100011F422EB00C000917800009179000217DE
:1004200018F003E0002E09C000E0001611F00A9455
:1004300004C000E008BD0093B40000C02F911F91DC
:100440000F91FFBE18951895189518951895189541
:100450001895FFB60F930091C6000B3411F4B1E06C
:10046000A0E2A03320F40D93AB3209F491600F9118
:10047000FFBE189518951895189518951895189504
:10048000189518951895189518953F93AF93BF93A5
:10049000B0E0A0E02053203031F034E6A30F30E08C
:1004A000B31F2A95D1F71053103019F01A961A95E8
:1004B000E9F70053A00F00E0B01F1B2F0A2FBF91D8
:1004C000AF913F91089510E010937A0010917C0055
:1004D000107F102B10937C0000E000937B0005EC54
:1004E00000937A0000917A0006FDFCCF009178001D
:1004F000109179000895011710F0201700F0089569
:100500006F937F93712F602F621B730B28F0712FF5
:10051000602F461B570B00F07F916F9108954F930A
:100520005F936F934427552760E1000F111F441F0D
:10053000551F4217530718F00395421B530B6A953A
:10054000A1F75F934F932F913F916F915F914F91DF
:1005500008951F9317B5011708F0012F08BD1F91CB
:1005600008951F931091B300011708F0012F009315
:10057000B4001F9108950F921F923F93019F112D78
:10058000002D30E0CCDF3F911F900F9008951F9316
:10059000F999FECF10E01FBB10E012BD81BD00BD78
:1005A000753A11F4FA9AF99A1F9108951F93F999DF
:1005B000FECF10E012BD81BDF89A00B51F910895DD
:1005C0001F932F932BE11BE51A95F1F72A95D9F785
:0A05D0000A95C1F72F911F910895BD
:00000001FF
